:10000000E0280408A2008316051183120930A3001A
:1000100003101120A20CA30B0928031411200314B0
:10002000DB280318162800000515182805111828C4
:100030000030A10062307928B31329080319B317DF
:100040000530A8002730A300103032200330A30071
:10005000E8303220A30164303220A3010A3032207C
:1000600024083928A2002508A1002408A000A42003
:100070002008A000A8030319B31329080319432873
:100080002802031808002008031DB313B31B08003F
:10009000303ED62883178001840AFF3E031D4B287B
:1000A000DB28031783168C010C1483120C0803172A
:1000B0008D0ADB28030103178C0083168C010C15B5
:1000C00055308D00AA308D008C148C1865280C11C9
:1000D00083128D0ADB28A301A200FF30A207031CB4
:1000E000A307031CDB280330A100E33079206D282F
:1000F000A101F43EA000A109FE30031C8228A00744
:1001000003187F28A0076400A10F7F280000201893
:10011000892820188B280800A20003309428A20008
:1001200006309428A2000530A80023082102031DF0
:100130009B282208200204300318013003190230E2
:100140002805031DFF30DB28A501A4011030A600FF
:10015000210DA40DA50D2208A4022308031C230FC2
:10016000A5020318BA282208A40723080318230F9E
:10017000A5070310A00DA10DA60BA8282008DB28B9
:100180001030A800A101A001A70CA60C031CCE28CA
:100190002208A00723080318230FA107A10CA00C15
:1001A000A50CA40CA80BC4282408DB288400310863
:1001B0008A0030088200831303138312640008004E
:1001C00083167E308F0007309C009D0183129701BB
:1001D000900183169001E3308500FF308600831282
:1001E00083169F0183129F0183169B012030840098
:1001F000603083128A014B20A030840050308A0185
:100200004B201030840060308A014A2090308400F6
:1002100060308A014A2064308A016B200130C200BC
:10022000C3010930BE00BF0132308A016B203E0895
:1002300003178D0003138A015120B800B901323031
:100240008A016B20FF30A000A1013908A300380803
:100250008A0192208A11031D2F29B801B901B80A19
:100260000319B90A3E0803178D00031338088A01E1
:100270005B2032308A016B2085110515831605112C
:10028000323083128A016B200D308A0102200A303D
:100290008A0102200D308A0102200A308A010220E0
:1002A00032308A016B20420803178D0003138A0144
:1002B0005120C000C101FF30A000A1014108A300EE
:1002C00040088A0192208A11031D73291430C0004E
:1002D000C101420803178D00031340088A015B2007
:1002E00032308A016B204008A6004108A7000A307E
:1002F000A200A3018A01C020C0002508C1004D3022
:100300008A01022055308A0102204C308A010220E5
:1003100054308A01022059308A0102204B308A0170
:10032000022045308A01022059308A010220203003
:100330008A01022056308A01022045308A010220BB
:1003400052308A01022053308A01022049308A014A
:1003500002204F308A0102204E308A0102202030D4
:100360008A01022031308A0102202E308A010220C7
:1003700030308A0102200D308A0102200A308A01C1
:1003800002200D308A0102200A308A010220423008
:100390008A01022059308A01022020308A0102207D
:1003A00052308A01022055308A01022049308A01E8
:1003B000022020308A01022043308A01022041308D
:1003C0008A01022042308A01022052308A01022032
:1003D00041308A0102204C308A0102200D308A010E
:1003E00002200A308A0102200D308A0102200A30E0
:1003F0008A0102204C308A0102204F308A010220FB
:1004000047308A01022020308A01022023308A01ED
:10041000022020308A010220A9013808A4003908EE
:10042000A5000130B000B1018A011C200D308A0105
:1004300002200A308A0102200D308A0102200A308F
:100440008A01022052308A01022041308A010220B2
:1004500054308A01022045308A01022020308A016E
:1004600002203D308A01022020308A010220A901A9
:100470004008A4004108A5000130B000B1018A0184
:100480001C200D308A0102200A308A0102200D3022
:100490008A0102200A308A01022064008A11861D26
:1004A0009B2A64008A11861D572A8A01512A20300E
:1004B0008A01022045308A0102204E308A01022042
:1004C00054308A01022045308A01022052308A01CC
:1004D000022049308A0102204E308A010220473032
:1004E0008A01022020308A01022053308A01022032
:1004F00045308A01022054308A01022055308A0199
:10050000022050308A0102202E308A0102202E3033
:100510008A0102202E308A0102200D308A01022039
:100520000A308A0102200D308A0102200A308A0135
:1005300002208A11392C0D308A0102200A308A01EA
:10054000022020308A01022053308A0102205430D8
:100550008A01022041308A01022052308A010220A1
:1005600054308A01022049308A0102204E308A012B
:10057000022047308A0102202E308A0102202E30CC
:100580008A0102202E308A0102200D308A010220C9
:100590000A308A0102200D308A0102200A308A01C5
:1005A0000220851164008A11061CEF2A64008A115A
:1005B000061CEF2A31308A0102200D308A01022008
:1005C0000A308A01022008308506831685118312BD
:1005D0004108A30040088A016C208A01D62A6400E1
:1005E0008A11861C0C2B64008A11861C0C2B32305D
:1005F0008A0102200D308A0102200A308A0102207D
:10060000083085068316851183124108A30040082F
:100610008A016C208A01F32A64008A11061D292BA5
:1006200064008A11061D292B33308A0102200D3007
:100630008A0102200A308A010220083085068316CA
:10064000851183124108A30040088A016C208A01A9
:10065000102B64008A11861D462B64008A11861DAA
:10066000462B34308A0102200D308A0102200A30E4
:100670008A010220083085068316851183124108FD
:10068000A30040088A016C208A012D2B64008A1186
:10069000061E632B64008A11061E632B35308A0107
:1006A00002200D308A0102200A308A01022008301F
:1006B00085068316851183124108A30040088A012C
:1006C0006C208A014A2B64008A11861E802B6400EC
:1006D0008A11861E802B36308A0102200D308A0155
:1006E00002200A308A01022008308506831685110F
:1006F00083124108A30040088A016C208A01672BFD
:1007000064008A11061F9D2B64008A11061F9D2B11
:1007100037308A0102200D308A0102200A308A0116
:100720000220083085068316851183124108A30034
:1007300040088A016C208A01842B64008A11861F7C
:10074000BA2B64008A11861FBA2B38308A01022026
:100750000D308A0102200A308A0102200830850605
:100760008316851183124108A30040088A016C207A
:100770008A01A12B64008A11051FD72B64008A11FE
:10078000051FD72B39308A0102200D308A01022043
:100790000A308A01022008308506831685118312EB
:1007A0004108A30040088A016C208A01BE2B640026
:1007B0008A11851FF72B64008A11851FF72B3130B2
:1007C0008A01022030308A0102200D308A01022085
:1007D0000A308A01022008308506831685118312AB
:1007E0004108A30040088A016C208A01DB2B6400C9
:1007F0008A11051C172C64008A11051C172C313036
:100800008A01022031308A0102200D308A01022043
:100810000A308A010220083085068316851183126A
:100820004108A30040088A016C208A01FB2B640068
:100830008A11851C372C64008A11851C372C3130B5
:100840008A01022032308A0102200D308A01022002
:100850000A308A010220083085068316851183122A
:100860004108A30040088A016C208A011B2C8A01E0
:10087000D12A0830850683168511FA3083128A0141
:100880006B2064008A11061C682C0530C007031811
:10089000C10A52308A01022041308A0102205430BC
:1008A0008A01022045308A0102203D308A0102205F
:1008B000A9014008A4004108A5000130B000B10121
:1008C0008A011C200D308A0102200A308A01022090
:1008D00064008A11861C912C0530C0020030031C74
:1008E000013EC10252308A01022041308A010220B9
:1008F00054308A01022045308A0102203D308A01AD
:100900000220A9014008A4004108A5000130B00060
:10091000B1018A011C200D308A0102200A308A01AF
:1009200002204008A0004108A100A3010A308A016A
:100930008C208A11031D9F2C0A30C000C101400881
:10094000A0004108A1000930A300F6308A018F20E1
:100950008A11031DAF2CF630C0000930C1006400BD
:100960008A11061DC32C64008A11061DC32C083091
:1009700085068316851183124108A30040088A0169
:100980006C208A01B32C64008A11861D552D6400E9
:100990008A11861DCD2C8A01C72C4008A000410871
:1009A000A1000A30A200A3018A01A420C0002108EE
:1009B000C100420803178D00031340088A015B2021
:1009C00032308A016B204008A6004108A7000A3097
:1009D000A200A3018A01C020C0002508C100523036
:1009E0008A01022041308A01022054308A0102200B
:1009F00045308A01022020308A010220A9014008E6
:100A0000A4004108A5000130B000B1018A011C20FA
:100A100020308A01022053308A01022041308A01AD
:100A2000022056308A01022045308A0102204430DB
:100A30008A01022020308A01022021308A0102200E
:100A400020308A0102200D308A0102200A308A01FA
:100A5000022020308A01022053308A0102205430C3
:100A60008A01022041308A01022052308A0102208C
:100A700054308A01022049308A0102204E308A0116
:100A8000022047308A0102202E308A0102202E30B7
:100A90008A0102202E308A0102200D308A010220B4
:100AA0000A308A0102208A01D12A8A01392C630086
:040AB0008A01572D33
:02400E00383F39
:00000001FF
